:020000040000FA
:02000000EE28E8
:08000800A200030EA1008030EC
:100010008107A620B42080302C0203190617AC0AF1
:10002000AC08031D1B280613AD0A3C302D02031D2E
:100030001B28AD01C22023200B111E28210E830096
:10004000A20E220E0900A003031D28280430A000E0
:1000500001302002031D31280E3085002308A7003F
:100060004C2802302002031D3A280D308500240858
:10007000A7004C2803302002031D43280B308500C5
:100080002508A7004C2804302002031D4C28073007
:1000900085002608A7004C2800302702031D55289C
:1000A0000611861106128612080001302702031D70
:1000B0005E280615861106128612080002302702F5
:1000C000031D6728061186150612861208000330E4
:1000D0002702031D702806158615061286120800D1
:1000E00004302702031D7928061186110616861290
:1000F000080005302702031D822806158611061602
:100100008612080006302702031D8B28061186156B
:1001100006168612080007302702031D94280615CC
:10012000861506168612080008302702031D9D2832
:100130000611861106128616080009302702031DD3
:100140000800061586110612861608002918AE2822
:100150000618080029143230AA000800AA03031D5B
:1001600008002910E12008002818BC28861808007B
:1001700028143230AB000800AB03031D0800281020
:10018000CE200800A60A0A302602031D0800A60198
:10019000A50A06302502031D0800A501033024022C
:1001A000031DD92802302302031DD928A401A3016D
:1001B0000800A40A0A302402031D0800A401A30AAF
:1001C0000800A60A0A302602031D0800A601A50A97
:1001D00006302502031D0800A50108008312031341
:1001E0008501860107309F008316031328308100A4
:1001F000103085008330860083120313A0308B00FB
:1002000085018101A301A401A501A601A701AC01FB
:10021000AD010430A000A901A8013230AA00AB0052
:040220001129112966
:02400E00223F4F
:00000001FF
